:0300000002343E89
:0C343E0078FFE4F6D8FD75816A02348541
:100F7B0020000A3C2E2E2E3E004950436F6E6E65AC
:100F8B0063745245510A004950436F6E6E6563742A
:100F9B00000A49504E6F41434B210A003E432C56E9
:100FAB002C43432CC0E4E0EFF2E5F020D1E8EDEA6E
:100FBB00EEEC49500A003E432C4D41432C25303278
:100FCB0062583A25303262583A25303262583A2507
:100FDB00303262583A25303262583A2530326258F4
:100FEB002C4D414320E0E4F0E5F10A003E432C5642
:100FFB0045522C20332E3220EEF220257320257300
:10100B002CC2E5F0F1E8FF20495020ECEEE4F3EBC5
:10101B00FF0A004A756E20303820323031310030F3
:10102B00393A30343A3132003E432C4C442C505236
:10103B004F473A2020202020202020202020202035
:10104B002020202020202020202020202020202095
:10105B002020202020202020202020202020202085
:10106B002020202020202020202020202020202075
:10107B0020202020202020202CC4E0F2E020EFF0C4
:10108B00EEF8E8E2EAE828F4E0E9EB290A003E2A68
:10109B002C312CCEF1EDEEE2EDFBE520EFE0F0E0B4
:1010AB00ECE5F2F0FB20F1E5F2E5E2EEE3EE20E811
:1010BB00EDF2E5F0F4E5E9F1E00A003E412C4130B8
:1010CB00312C2562752E2562752E2562752E2562B3
:1010DB00752C495020E0E4F0E5F120E0E4E0EFF27C
:1010EB00E5F0E00A003E412C4130322C2562752E92
:1010FB002562752E2562752E2562752C495020E0D0
:10110B00E4F0E5F120EEF1ED2E20F1E5F0E2E5F073
:10111B00E00A003E412C4130332C2562752E2562AE
:10112B00752E2562752E2562752C495020E0E4F052
:10113B00E5F120F0E5E72E20F1E5F0E2E5F0E00A3D
:10114B00003E412C4130342C2562752E2562752EC4
:10115B002562752E2562752CCCE0F1EAE020F1E5D5
:10116B00F2E80A003E412C4130352C2562752E25C4
:10117B0062752E2562752E2562752CD8EBFEE70A5B
:10118B00003E2A2C312CC4EEEF2E20EFE0F0E0ECE9
:10119B00E5F2F0FB20F1E5F2E5E2EEE3EE20E8ED1F
:1011AB00F2E5F0F4E5E9F1E00A003E422C53303170
:1011BB002C2562752CC6E4E0F2FC20E7E0EFF0EEA4
:1011CB00F1E020F1EEE5E4E8EDE5EDE8FF20EEF2ED
:1011DB0020F1E5F0E2E5F0E00A003E422C5330321C
:1011EB002C2562752CCEE1ECE5ED20F120F1E5F03C
:1011FB00E2E5F0EEEC20E1E5E720EAE2E8F2E0EDF3
:10120B00F6E8E90A003E422C5330332C2562752C4C
:10121B00CFE5F0E5E7E0EFF3F1EA20EFF0E820EFC0
:10122B00EEF2E5F0E520F1E2FFE7E820F120F1E551
:10123B00F0E2E5F0EEEC0A003E422C5330382C2560
:10124B0062752CCCE5E4EBE5EDEDFBE92049502094
:10125B00EAE0EDE0EB28E7E0E4E5F0E6EAE020E4A5
:10126B00EE203520F1E5EA290A003E454E440A00FE
:10127B000A44756D705820202020203030203031EA
:10128B00203032203033203034203035203036209F
:10129B003037203038203039203041203042203058
:1012AB0043203044203045203046000A3A003A2093
:1012BB00000A000A44756D70442020202020303035
:1012CB002030312030322030332030342030352064
:1012DB003036203037203038203039203041203024
:1012EB0042203043203044203045203046004572A8
:1012FB0072206B657900526420656570726F6D0AA0
:10130B00005264204D454D0A00526420436F6465C2
:10131B000A00577269746520436F64650A0044655F
:10132B006275674950204F4E0A00446562756749E4
:10133B0050204F46460A00446562756755736572C7
:10134B00204F6E0A00446562756755736572204FB6
:10135B0046460A0044656275674D7367204F6E0AF7
:10136B000044656275674D7367204F46460A00431C
:10137B006F6E666967206C6F636B210A0057722072
:10138B00656570726F6D0A00205361766520656527
:10139B0070726F6D210A00457272204D414321001E
:1013AB004C6F61643E3E002A00CEF8E8E1EAE00AA9
:1013BB0000202D202575282575290A003C41303148
:1013CB003D003C4130323D003C4130333D003C411F
:1013DB0030343D003C4130353D003C21003C533026
:1013EB00313D003C5330323D003C5330333D003CEB
:1013FB005330353D003C5330383D003C5330363D87
:01140B0000E0
:063E6600010B0001090040
:103E5600C28E438910758BFF758DB7D2ABD28E2279
:03001B000233AEFF
:1033AE00C0E0C083C082C0D0C28E758BFF758DB752
:1033BE0020060675A61E75A6E10509D202E50B606C
:1033CE0002050B050EE50E540F7051E50AD394015C
:1033DE004002150AD20EE50E543F7012D2009066CE
:1033EE008EE0600A04F0E0D394B44002D2069066F8
:1033FE0087E0600204F0906104E0600214F09066D1
:10340E008FE0D394014003E014F0300502050CE583
:10341E000DD394644004D2068002050DE508D394C2
:10342E000140021508D28ED0D0D082D083D0E032A7
:1008EF00C291C290D2B5C20B7D027C007F07123E2F
:1008FF00058F4AE54A646060097D017F60123D59AA
:10090F00D20BE4FDFC7F0B123E058F4AE54A30E621
:10091F00097D04E4FF123D7DD20B7D017C007F0732
:10092F00123E058F4AE54A7008FD7FFF123D59D2EE
:10093F000B300B03126000C288C2A8C2AA758900CF
:10094F001237EA90633FE0B4FA06A3E064CE607B0F
:10095F00E4F54A7437254AF582E43463F583E4F00D
:10096F00054AE54AB443EC90633F74FAF0A374CEA2
:10097F00F0A374CCF0906345740AF0E4A3F0A304E1
:10098F00F0A3F090633B74FFF0A3F0A3F0E4A3F0A7
:10099F009063567403F0E4F54AE54A2401FFE4330B
:1009AF00FE7437254AF582E43463F583E0FD123D8A
:1009BF0035054AE54AC3944340DFE4F5A775A61E03
:1009CF0075A6E1907FF0F0A3F080FE90634A740368
:1009DF00F0A374CCF0E4906349F090668CF0A3F030
:1009EF00122E05C2B51239BAC206123B9ED20BC2E5
:1009FF000DC20C9065777408F09062B57424F0E422
:100A0F00A3F090633FE09062B7F0906340E0906294
:100A1F00B8F0906341E09062B9F0906342E0906269
:100A2F00BAF0906343E09062BBF0906344E0906251
:100A3F00BCF0750A01E4906578F0C207C208C209DC
:100A4F00C20A123DA1200B19AF4A7E007D03122E60
:100A5F00EBE4FF1232FE7E0F7F7BE4FBFDFC1229DD
:100A6F001D90668EE060037401F0E4906104F0F570
:100A7F000C906576F0F50D123E5675A70775A61EFC
:100A8F0075A6E1D2AFE4F50D906104E07003121783
:100A9F006890668FE06401701D9080007410F09074
:100AAF0080A874FFF0A3F0A3F0A3F0E490668FF09A
:100ABF00D20BC20CC20D908008E0F54A30E405D28B
:100ACF00077410F0E54A30E508D2099080087420C9
:100ADF00F0E54A30E608D2089080087440F0E50C43
:100AEF00C394034019908002E4F0908001F090804D
:100AFF0000F0E50C94064006E4F50C123B9E908046
:100B0F00A0E070031238E29080B8E07003123868EA
:100B1F009080D0E07003123B42908000E070133061
:100B2F000710122A24906332EFF0D394004003127F
:100B3F000036908002E07006908000E06005D205DC
:100B4F00020A94C205E4F50C906104E06003020A06
:100B5F0094200B12906579E0600C7E0F7F7D122D33
:100B6F001DE4906579F030091212252A906332EF57
:100B7F00F0D394004005E0FF12002F200803020D70
:100B8F0018122222906332EFF07003020A949063DE
:100B9F0076E054BF247F7003020C73147003020CB1
:100BAF004B24026003020CBA200B077E0F7F8412C6
:100BBF002D1D200F03020D1890634EE070069063F9
:100BCF0052E06067906683E0FF90634EE0B50724C4
:100BDF00906684E0FE90634FE0B50618906685E05E
:100BEF00FE906350E0B5060C906686E0FE90635170
:100BFF00E06E6037906352E06F6003020D189066ED
:100C0F0084E0FF906353E06F6003020D18906685D8
:100C1F00E0FF906354E06F6003020D18906686E06A
:100C2F00FF906355E06F6003020D18C20390657863
:100C3F007401F0120022750A01020D1890668EE001
:100C4F0060037401F090667BE0FF906378E06F6063
:100C5F0003020D1890667BE004F0E4F50A906576C8
:100C6F00F0020D18300303020D18906345E0700376
:100C7F00020A949062B4E06008906356741EF0808C
:100C8F00069063567403F0123E6DD203E4F50A909A
:100C9F006576F090668704F0E490667AF0A3F02012
:100CAF000B677E0F7F92122D1D805E90668EE06027
:100CBF00037401F0300352906376E020E74B9063AA
:100CCF0078E0FF90667AE0FE6F600D906682E070CC
:100CDF0007EE146F7033801390667AE004F0906320
:100CEF0032E0FFD3940440031227E6906000748231
:100CFF00F0A37401F0906378E0906002F07E607F63
:100D0F00007D03123551020A94200303020E3BE5C6
:100D1F000A706E123950EF60237E647F769064778D
:100D2F00E02404FD123551906682E07009906356FD
:100D3F00E0F50A020A94E4F50A020A94906687E045
:100D4F00D3943C403C906682E070369062B4E07081
:100D5F003090668704F0120032E4906476F0A3744A
:100D6F0012F090667BE0906478F0A374FDF09061D0
:100D7F000563A20190647A63A2017F12121F708033
:100D8F0098123E3C8F4AE54AB40115906000748377
:100D9F00F0E4A3F07E607F007D02123551020A94C9
:100DAF00E54AD39401401C9060007483F0A3740152
:100DBF00F0E54A24FEA3F07E607F007D03123551DB
:100DCF00020A94E50A64016003020A94906576E0D2
:100DDF0004F0200B077E0F7F9C122D1D906576E08F
:100DEF00FFD39401400B906356E0941E5003E00430
:100DFF00F0EFC39405400DC203E4906578F0120044
:100E0F0022020A947C667D8390634AE0FAA3E0FB9A
:100E1F007F021236E27E647F76906477E02404FDD1
:100E2F00123551906356E0F50A020A94E50A6401FF
:100E3F006003020A94906578E014604624FE6042D5
:100E4F00147003020F2E24046003020A94E4F50CBD
:100E5F00200F139065787404F0906576E05401F0DC
:100E6F00750A01020A949080027410F0E49065787C
:100E7F00F090657604F0750A1290668374FFF002A5
:100E8F000A94906683E07003020F18906476748062
:100E9F00F09064787401F0E4A3F0A304F0A374302D
:100EAF00F0A3747BF0E4F54A747D254AF582E434AF
:100EBF0064F583747DF0747E254AF582E43464F51D
:100ECF0083E4F0E54A2407906477F07C667D839095
:100EDF00634AE0FAA3E0FB7F021236E27E647F767C
:100EEF00E54A2409FD123551906682E0601B123EDF
:100EFF006DD203E4F50A906576F090668704F0E40E
:100F0F0090667AF0A3F0020A94300F07E4906578A8
:100F1F00F080069065787404F0750A12020A9490B6
:100F2F0080027410F0750A03906576E06401FFF09B
:100F3F009065787401F0EF7019906352E06013FCC4
:100F4F00A3E0FDA3E0FEA3E0FF906683121B120255
:100F5F000A9490634EE0FCA3E0FDA3E0FEA3E0FF44
:0B0F6F00906683121B12020A9480FEA1
:010F7A002254
:10003600906377E0B444047F0180027F009063768A
:10004600E0B447047E0180027E00EE5F604A906362
:100056003FE0906378F0906340E0906379F09063BE
:1000660041E090637AF0906342E090637BF09063A6
:1000760043E090637CF0906344E090637DF090638E
:10008600777452F09062AE63A2019080A863A201D9
:100096007F06121F700208E5906332E0C394085091
:1000A600030208EE90633FE0FF906378E06F600321
:1000B6000208EE906340E0FF906379E06F60030210
:1000C60008EE906341E0FF90637AE06F60030208F8
:1000D600EE906342E0FF90637BE06F60030208EE00
:1000E600906343E0FF90637CE06F60030208EE904C
:1000F6006344E0FF90637DE06F60030208EE906367
:1001060077E06444701A9080A8E0B4FF139062AE62
:1001160063A2019080A863A2017F06121F7080105F
:100126009062B2E09080ACF09062B3E09080ADF067
:1001360090668EE060037401F090668F7464F090B0
:1001460063777452F0906376E0646D600302028810
:100156007BFF7A0F79A712146E7BFF7A0F79C19015
:10016600633FE0F553A3E0F554A3E0F555A3E0F5AE
:1001760056A3E0F557A3E0F55812146E7553FF75B4
:10018600541075551E7556FF75571075582A7BFF06
:100196007A0F79F712146E7BFF7A10793312146E88
:1001A6007BFF7A10799912146E7BFF7A1079C690CC
:1001B6006345E0F553A3E0F554A3E0F555A3E0F558
:1001C6005612146E7BFF7A1079F090634EE0F55369
:1001D600A3E0F554A3E0F555A3E0F55612146E7BA3
:1001E600FF7A11791E906352E0F553A3E0F554A30C
:1001F600E0F555A3E0F55612146E7BFF7A11794CA3
:1002060090633BE0F553A3E0F554A3E0F555A3E076
:10021600F55612146E7BFF7A11796F906337E0F50D
:1002260053A3E0F554A3E0F555A3E0F55612146E7A
:100236007BFF7A11798C12146E7BFF7A1179B5A245
:100246000FE433F55312146E7BFF7A1179E590664D
:1002560082E0F55312146E7BFF7A12791090668E47
:10026600E0F55312146E7BFF7A1279439062B4E084
:10027600F55312146E12317C7BFF7A1279751214C3
:100286006E22906376E0644C70737E127F7BFBFD7A
:10029600FC12291D90637EE0F54BA3E0F54CE4F5D6
:1002A6004EE54B906380F0A3E54CF07E127FB67C62
:1002B600637D807B0212291DE4F54D854C82854BBA
:1002C60083E0FF7480254DF582E43463F583EFF017
:1002D600054CE54C7002054B054DE54DB410DC7E32
:1002E600127FB97C637D807B1012291D054EE54E79
:1002F600C3941040AC7E127FBC122D1D22906376F3
:10030600E0646C7060F54F7E127FBEFBFDFC122927
:100316001DE4F54EE4906380F0A3E54FF07E127F76
:10032600B67C637D807B0212291DE4F54DA84FE65D
:10033600FF7480254DF582E43463F583EFF0054FB5
:10034600054DE54DB410E67E127FB97C637D807B5A
:100356001012291D054EE54EC3940840B77E127F44
:10036600BC122D1D22906376E0644B7061F54D74CE
:1003760068254DF582E43463F583E06032746825C0
:100386004DF582E43463F583E0F460237468254D0B
:10039600F582E43463F583E0FF747E254DF582E44F
:1003A6003463F583E0B50710054DE54DB408C090FC
:1003B60061047432F00208E59063767421F0300B24
:1003C600030208E57E127FF9122D1D0208E59063EF
:1003D60076E0B4521A200B077E137F01122D1D9072
:1003E60063767472F07E637F767D081234CA22903B
:1003F6006376E064497045200B077E137F0C122D4F
:100406001D90637EE0F54BA3E0F54CE4F54D854C7D
:1004160082854B83E0FF7480254DF582E43463F5D5
:1004260083EFF0054CE54C7002054B054DE54DB4E8
:1004360080DC7E637F767D8A1234CA22906376E002
:1004460064437046200B077E137F14122D1D9063A4
:100456007EE0F54BA3E0F54CE4F54D854C82854BEB
:1004660083E493FF7480254DF582E43463F583EFCE
:10047600F0054CE54C7002054B054DE54DB480DBAF
:100486007E637F767D8A1234CA22906376E0645A50
:100496007053200B077E137F1D122D1D90637EE087
:1004A600F54BA3E0F54C7C637D807B80AF4CAE4B77
:1004B600123C79E4F54D854C82854B83E493FF74B9
:1004C60080254DF582E43463F583EFF0054CE54C69
:1004D6007002054B054DE54DB480DB7E637F767D6E
:1004E6008A1234CA22906376E06444600302057C73
:1004F60090637EE0FF644470030208E5EFB4310CBC
:10050600C20B7E137F29122D1D0208E590637EE043
:10051600B4300CD20B7E137F35122D1D0208E590E8
:10052600637EE0B4320CD20C7E137F42122D1D0284
:1005360008E590637EE0B4330CC20C7E137F501244
:100546002D1D0208E590637EE0B4340CD20D7E13B7
:100556007F5F122D1D0208E590637EE0B4350CC264
:100566000D7E137F6C122D1D0208E590637EE0FF61
:1005760012001E0208E5906104E07013200B077E4E
:10058600137F7A122D1D9063767421F00208E59090
:1005960061047432F0906376E0FFB45104C2AF8018
:1005A600FEEF64577045200B077E137F88122D1DC2
:1005B60090637FE0906332F0E4F54D906332E0FFA4
:1005C600E54DC39F40030208E57480254DF582E49E
:1005D6003463F583E0FF90637EE0254D24ADF5821C
:1005E600E43461F583EFF0054D80D0906376E064E6
:1005F60053600302069F200B077E137F93122D1D67
:1006060090633FE0FF9061B6E06F703C906340E01E
:10061600FF9061B7E06F7030906341E0FF9061B882
:10062600E0B50724906342E0FF9061B9E0B5071892
:10063600906343E0FF9061BAE0B5070C906344E035
:10064600FF9061BBE06F60169063767421F0300B0B
:10065600030208E57E137FA2122D1D0208E5E4F5CC
:100666004DE4F50DAF4DFE74AD254DF582E43461D4
:10067600F583E0FD123D35054DE54DC394FE40E1A1
:10068600C2AFE4907FF0F0A3F0907FFD74AAF0A3D0
:1006960074FFF0A37455F080FE906376E0644F70AB
:1006A6005A90637EE0F54BA3E0F54CE54C454B7064
:1006B6000A200B077E137FAB122D1D200B077E131E
:1006C6007FB2122D1DE4F54D7480254DF582E4347C
:1006D60063F583E0854C82854B83F0054CE54C70D1
:1006E60002054B054DE54DB480DE90668DE0248015
:1006F600F090668CE03400F00208E5906376E064E2
:1007060045707490637EE0FEA3E0FF907FF0EEF00C
:10071600A3EFF0D39400EE94044038907FF0E0FE0F
:10072600A3E0FF90668CE0FCA3E0FD9FEC9E4023D7
:10073600E42FFFEE3401FED3ED9FEC9E5015C2AFC1
:10074600907FFD74AAF0A374FFF0A37455F0E4F54E
:10075600A780FE7E137FB4122D1D7BFF7A1379BC12
:10076600907FF0E0F553A3E0F55490668CE0F555E4
:10077600A3E0F55612146E906376E064656003029A
:1007860008EE90637EE0FFA3E0907FF0CFF0A3EF4A
:10079600F0E4F54BF54CD3907FF1E0954C907FF06B
:1007A600E0954B4020E4F50D254CFFE54B3401FE6A
:1007B600854C82854B83E0FD123D35054CE54C703A
:1007C60002054B80D17E137FC71235D8EF4E6020CD
:1007D600120003906345EFF0120003906346EFF0BA
:1007E600120003906347EFF0120003906348EFF0A6
:1007F6007E137FCD1235D8EF4E6020120003906332
:100806004EEFF012000390634FEFF0120003906377
:1008160050EFF0120003906351EFF07E137FD31276
:1008260035D8EF4E6020120003906352EFF01200AD
:1008360003906353EFF0120003906354EFF012003D
:1008460003906355EFF07E137FD91235D8EF4E60D3
:100856002012000390633BEFF012000390633CEF1D
:10086600F012000390633DEFF012000390633EEF39
:10087600F07E137FDF1235D8EF4E60201200039012
:100886006337EFF0120003906338EFF01200039025
:100896006339EFF012000390633AEFF0E4F54DE4AC
:1008A600F50DE54D2401FFE433FE7437254DF58241
:1008B600E43463F583E0FD123D35054DE54DC39403
:1008C6004340DCC2AFE4907FF0F0A3F0907FFD746C
:1008D600AAF0A374FFF0A37455F0E4F5A780FE7E9A
:0808E600637F767D081234CA1D
:0108EE0022E7
:103C4100AE07EEC39430400BEED394395005EE2409
:103C5100D0FF22EEC39461400BEED394665005EE83
:103C610024A9FF22EEC39441400BEED394465005A4
:083C7100EE24C9FF22AF062278
:103E22009062ADE004F070069062ACE004F0906243
:0A3E3200ACE0FEA3E0FF123DE82221
:10000300123E22123C41EFC454F0FEC006123E22BF
:08001300123C41D0E02FFF2256
:103AE500E4906A11F0123E22906A12EFF0C394300E
:103AF5004018E0FFD394395011906A11E02405F580
:103B050082E43461F583EFF08011906A11E02405B9
:103B1500F582E43461F583E4F0800C906A11E004E9
:103B2500F0E0D3940840BE754F0075500075510004
:0C3B3500E4F5527B017A61790512207ED4
:013B41002261
:0435D8008E508F5131
:1035DC009062ACE4F0A374FFF0123E22EF606EF444
:1035EC00606B855182855083E493B507EC7552016D
:1035FC00E5512552F582E43550F583E4936025902E
:10360C0062ADE02552FF9062ACE03400FE123DE862
:10361C00E5512552F582E43550F583E493B5070462
:10362C00055280CCE5512552F582E43550F583E402
:10363C009370A6E55224FFFFE434FFFE9062ADE0E8
:10364C002FF09062ACE03EF07E007F0122E4FEFFA2
:01365C00224B
:102E05007E137FE51235D8EF4E70037F01227E13C6
:102E15007FE81235D8EF4E600C123E22EF24D02405
:102E2500FF920F8002D20F7E137FEE1235D8EF4E40
:102E3500600C123E22EF24D0906682F08005E4906B
:102E45006682F07E137FF41235D8EF4E600C123E89
:102E550022EF24D090668EF08005E490668EF07E99
:102E6500137FFA1235D8EF4E600C123E22EF24D0B4
:102E750024FF92018002C2017E147F001235D8EF33
:102E85004E600C123E22EF24D09062B4F08005E42F
:102E95009062B4F090633F63A20190667C63A201E7
:102EA5007F06121F7030013B7E147F061235D8EF66
:102EB5004E603012000390667CEFF01200039066BE
:102EC5007DEFF012000390667EEFF012000390662E
:102ED5007FEFF0120003906680EFF012000390661A
:062EE50081EFF07F0022E6
:103BF800906577E0C3947C40027F0A906577E0FE89
:103C080004F074B52EF582E43462F583EFF0BF0A50
:103C180027906577E0FF04F074B52FF582E43462ED
:103C2800F583E4F0906577E0FF12365D9065777470
:093C380008F09062B6E004F022ED
:103B9E009080007480F090633763A201F583F58204
:103BAE0063A2017F08121F7090633F63A201908091
:103BBE008863A2017F0A121F709080927407F0A38F
:103BCE0074D0F0A37406F0906349E0FF9080B1F0DA
:103BDE009080E1EFF09080957455F0A3F090800006
:0A3BEE007401F090800974F0F022D9
:1038E200908009E04410F09080A0E070609080A188
:1038F2007482F09080A874FFF0A3F0A3F0A3F07F8D
:10390200039080AEEFF0A374CBF09080007402F0CD
:10391200906A05121B1E00000000906A05E090806C
:1039220040F0906A06E0908041F0906A07E0908053
:1039320042F0906A08E0908043F0A3E4F0A3F0A381
:0D394200F0A3F0908018F0A3F0A3F0A3F024
:01394F002255
:103B4200908009E04440F09080D17482F07F03902D
:103B520080DEEFF0A374CCF09080027402F0906AE1
:103B620009121B1E00000000906A09E0908058F0C4
:103B7200906A0AE0908059F0906A0BE090805AF0C7
:103B8200906A0CE090805BF0A3E4F0A3F0A3F0A3B2
:0B3B9200F0908030F0A3F0A3F0A3F04F
:013B9D002205
:10386800908009E04420F09080B8E0706C9080B9B6
:103878007482F07F039080C6EFF07FCDA3EFF07FD6
:10388800039080C4EFF0A374CDF09080C074FFF073
:10389800A3F0A3F0A3F09080017402F0906A0D12D7
:1038A8001B1E00000000906A0DE090804CF0906AAA
:1038B8000EE090804DF0906A0FE090804EF0906A94
:1038C80010E090804FF0A3E4F0A3F0A3F0A3F090F1
:0938D8008024F0A3F0A3F0A3F09A
:0138E10022C4
:1036E2008C4B8D4CA907EAFDE975F018A424ACFFB8
:1036F200E5F034808F82F583EDF0EBFDE975F0188B
:10370200A4FFAEF024ACFBEE34808B82F583A3EDF4
:10371200F0854C828C83E0FDEF24A8FFEE3480FE1E
:103722008F82F583EDF0854C828C83A3E08F828EAD
:1037320083A3F0854C82854B83A3A3E0FDE975F05A
:1037420018A424A8FFE5F03480FE8F82F583A3A39A
:10375200EDF0854C828C83A3A3A3E08F828E83A39A
:04376200A3A3F0220B
:0634CA008D50AB07AA06BD
:1034D000908000E030E5079065797401F022906AF1
:1034E00005E0FCA3E0FDA3E0FEA3E0F5548E538DC0
:1034F000528C51AE02AF038E838F8263A201E553DB
:10350000540744C0F58385548263A201AF50121F53
:10351000E2E4FCFDFEE5542550F554EE3553F55339
:10352000ED3552F552EC3551F551908040E551F0B2
:10353000A3E552F0A3E553F0A3E554F090800074A6
:1035400020F0AF54AE53AD52AC51906A05121B122D
:013550002258
:063551008D4BAB07AA063A
:10355700908002E030E5079065797403F022906A65
:1035670009E0FCA3E0FDA3E0FEA3E0F54F8E4E8D3E
:103577004D8C4CAE02AF038E838F8263A201E54E62
:10358700540744D0F583854F8263A201AF4B121FC6
:10359700E2E4FCFDFEE54F254BF54FEE354EF54ECB
:1035A700ED354DF54DEC354CF54C908058E54CF02C
:1035B700A3E54DF0A3E54EF0A3E54FF0908002742C
:1035C70020F0AF4FAE4EAD4DAC4C906A09121B12B6
:0135D70022D1
:0232FE008F4BF4
:10330000908001E030E5099065797402F07F002239
:10331000906A0DE0FCA3E0FDA3E0FEA3E0F54F8E74
:103320004E8D4D8C4C90667C63A201E54E54074453
:10333000C8F583854F8263A2017F06121FF8E54F0F
:103340002406F54FE4354EF54EE4354DF54DE435A4
:103350004CF54C90657A63A201E54E540744C8F5DC
:1033600083854F8263A201AF4B121FF8E4FCFDFE80
:10337000E54F254BF54FEE354EF54EED354DF54D00
:10338000EC354CF54C90804CE54CF0A3E54DF0A3AA
:10339000E54EF0A3E54FF09080017420F0AF4FAE02
:0D33A0004EAD4DAC4C906A0D121B12AF4BA0
:0133AD0022FD
:102A24009081E0E0F54B054B054B054B054B054B01
:102A3400054B054B054B054B054B908010E0F54EBF
:102A4400A3E0F54FA3E0F550A3E0F5519081E1E058
:102A5400F54B054B054B054B054B054B054B054B02
:102A6400054B054B054B908014E0F552A3E0F5535C
:102A7400A3E0F554A3E0F555E554B55008E555B584
:102A840051037F0022E4F54BE554540744E0F583F9
:102A940085558263A20190637663A2017F081220A8
:102AA4002890637863A2019062AE63A2017F06124C
:102AB4001F70906376E0F54CA3E0F54DE4F54B9080
:102AC4006376E0702AA3E024F8F54BE554540744F8
:102AD400E0F58385558274082582F582E43583F513
:102AE4008363A20190637663A201AF4B122028AEE8
:102AF4004CE4FCFDE555254DF555E5543EF554ED06
:102B04003553F553EC3552F552908014E552F0A349
:102B1400E553F0A3E554F0A3E555F090800074402C
:032B2400F0AF4BC4
:012B2700228B
:102222009081E6E0F54B054B054B054B054B054B05
:10223200054B054B054B054B054B908028E0F54EB1
:10224200A3E0F54FA3E0F550A3E0F5519081E7E05C
:10225200F54B054B054B054B054B054B054B054B0C
:10226200054B054B054B90802CE0F552A3E0F5534E
:10227200A3E0F554A3E0F555E4F54BE554B5500A57
:10228200E555B55105C20802238EE554540744F0C2
:10229200F58385558263A20190637663A2017F086C
:1022A200122028906376E0F54CA3E0F54DE54D450C
:1022B2004C70099080027410F07F0022906683E0D7
:1022C200FFF46030906378E06F60030223559066FC
:1022D20084E0FF906379E06F7079906685E0FF900B
:1022E200637AE06F706D906686E0FF90637BE06FCB
:1022F2006031805F906378E0906683F0906379E06C
:10230200906684F090637AE0906685F090637BE05B
:10231200906686F090637CE0FFA3E090634ACFF082
:10232200A3EFF0906376E0702AA3E024F8F54BE582
:1023320054540744F0F58385558274082582F5824A
:10234200E43583F58363A20190637663A201AF4B08
:10235200122028AE4CE4FCFDE555254DF555E5541B
:102362003EF554ED3553F553EC3552F552AF51AEBF
:1023720050AD4FAC4EAB55AA54A953A852D3121B21
:102382000140099080027410F07F002290802CE5B9
:1023920052F0A3E553F0A3E554F0A3E555F0908085
:0623A200027440F0AF4B95
:0123A8002212
:10252A009081E3E0F54B054B054B054B054B054BFD
:10253A00054B054B054B054B054B90801CE0F54EB2
:10254A00A3E0F54FA3E0F550A3E0F5519081E4E054
:10255A00F54B054B054B054B054B054B054B054B01
:10256A00054B054B054B908020E0F552A3E0F5534F
:10257A00A3E0F554A3E0F555E4F54BE554B5500A4C
:10258A00E555B55105C20902267EE554540744E8CB
:10259A00F58385558263A20190600463A2017F0ED0
:1025AA0012203E906004E0F54CA3E0F54D90600CDB
:1025BA00E0FFF4604A90667CE0FEEF6E7077A3E07D
:1025CA00FF90600DE06F706D90667EE0FF90600E88
:1025DA00E06F706190667FE0FF90600FE06F70556A
:1025EA00906680E0FF906010E06F7049906681E02D
:1025FA00FF906011E06F703DE4906013F0800690E8
:10260A00601374FFF0906004E0702AA3E024F2F5EE
:10261A004BE554540744E8F583855582740E2582A8
:10262A00F582E43583F58363A20190600463A20115
:10263A00AF4B12203EAE4CE4FCFDE555254DF55559
:10264A00E5543EF554ED3553F553EC3552F552AF9A
:10265A0051AE50AD4FAC4EAB55AA54A953A852D364
:10266A00121B015006E54D454C700990800174100B
:10267A00F07F0022908020E552F0A3E553F0A3E515
:0E268A0054F0A3E555F09080017440F0AF4B82
:01269800221F
:042D1D008E508F51F4
:102D2100908000E030E5079065797401F022906AA7
:102D310005E0FCA3E0FDA3E0FEA3E0F5578E568D70
:102D4100558C54E557FFE5565407FEE42FF553EE35
:102D510034C0F552855382F5837423F00553E5534E
:102D6100700205525352C7F582855283740AF005E9
:102D710053E553700205525352C790633F63A2015A
:102D810085528385538263A2017F06121FE2740676
:102D91002553F553E43552F55285508385518263AD
:102DA100A20185528385538263A201121FC6E4FCEE
:102DB100FDFE906A05E0F8A3E0F9A3E0FAA3E02F95
:102DC100FFEE3AFEED39FDEC38FCEF2408FFE43E5E
:102DD100FEE43DFDE43CFC906A05121B12906A057D
:102DE100E0908040F0906A06E0908041F0906A07A0
:102DF100E0908042F0906A08E0908043F09080007B
:032E01007420F04A
:012E040022AB
:0A291D008E508F518C528D538B5455
:10292700908000E030E5079065797401F022906AA5
:1029370005E0FCA3E0FDA3E0FEA3E0F55A8E598D68
:10294700588C57E55AFFE5595407FEE42FF556EE24
:1029570034C0F555855682F5837423F00556E55640
:10296700700205555355C7F582855583740AF005DE
:1029770056E556700205555355C790633F63A2014C
:1029870085558385568263A2017F06121FE274066E
:102997002556F556E43555F555855083855182639F
:1029A700A20185558385568263A201121FC68F5BDC
:1029B700EF2556F556E43555F555E554601785521C
:1029C7008385538263A20185558385568263A2015D
:1029D700AF54121FE2E55B24082554F554FFE4FCCD
:1029E700FDFEE55A2FF55AEE3559F559ED3558F5EF
:1029F70058EC3557F557908040E557F0A3E558F068
:102A0700A3E559F0A3E55AF09080007420F0AF5A7F
:0C2A1700AE59AD58AC57906A05121B1266
:012A23002290
:062FCC008E4C8F4D8D4E6E
:102FD200908000E030E5079065797401F022906AF4
:102FE20005E0FCA3E0FDA3E0FEA3E0F5548E538DC3
:102FF200528C51E554FFE5535407FEE42FF550EE91
:1030020034C0F54F855082F5837423F00550E550A6
:103012007002054F534FC7F582854F83EBF0055081
:10302200E5507002054F534FC790633F63A201857D
:103032004F8385508263A2017F06121FE274062528
:1030420050F550E4354FF54F854C83854D8263A290
:1030520001854F8385508263A201AF4E121FE27435
:1030620008254EF54EFFE4FCFDFEE5542FF554EE27
:103072003553F553ED3552F552EC3551F5519080FB
:1030820040E551F0A3E552F0A3E553F0A3E554F077
:103092009080007420F0AF54AE53AD52AC51906AA0
:0430A20005121B12E6
:0130A6002207
:02365D008F6478
:10365F00908000E030E5079065797401F022906A60
:10366F0005E0FCA3E0FDA3E0FEA3E0F5688E678D07
:10367F00668C65E568FFE5675407FEE42FFFEE34BF
:10368F00C09062B563A201F5838F8263A201AF641C
:10369F00121FE2E4FCFDFEE5682564F568EE356770
:1036AF00F567ED3566F566EC3565F565908040E5B7
:1036BF0065F0A3E566F0A3E567F0A3E568F09080F9
:1036CF00007420F0AF68AE67AD66AC65906A051206
:0236DF001B12BC
:0136E10022C6
:062EEB008E4E8F4FAB0577
:102EF100908000E030E5079065797401F022906AD6
:102F010005E0FCA3E0FDA3E0FEA3E0F5558E548DA2
:102F1100538C52E555FFE5545407FEE42FF551EE6D
:102F210034C0F550855182F5837423F00551E55184
:102F3100700205505350C7F582855083EBF005515F
:102F4100E5517002055090633F63A201855083856E
:102F5100518263A2017F06121FE274062551F551C9
:102F6100E43550F5505350C7E54E85518285508365
:102F7100F00551E551700205505350C7F582855057
:102F810083E54FF00551E551700205505350C7E5F7
:102F910055240AF555E43554F554E43553F553E415
:102FA1003552F552908040E552F0A3E553F0A3E588
:102FB10054F0A3E555F09080007420F0AF55AE5465
:0A2FC100AD53AC52906A05121B12CA
:012FCB0022E3
:103DE800A2AF921AC2AF438E2075D2028F828E8301
:0C3DF800E0FFE4F5D2538EDFA21A92AF78
:013E0400229B
:103D3500E5D220E0FBA2AF921AC2AF43D2028F8236
:103D45008E83EDF075D25063D250A21A92AFE5D2B0
:033D550020E0FB70
:013D58002248
:1037EA00E4FDED2401FFE433FE123DE874372DF5C4
:1037FA0082E43463F583EFF00DBD3FE6E4FDED248A
:10380A007FFFE433FE123DE8742D2DF582E4346126
:10381A00F583EFF0742D2DF582E43461F583E070C1
:10382A001B742D2DF582E43461F5837420F0742E17
:10383A002DF582E43461F583E4F080040DBD80BE89
:10384A00E49061ACF0FDEDFF7E00123DE874AD2D11
:0D385A00F582E43461F583EFF00DBDFEE969
:01386700223E
:023C79008B506E
:103C7B00A2AF921AC2AF85A25153A2FE8E838F823E
:103C8B0005A28C838D82740912206CE55053A2FE21
:103C9B0043A22012206E53A2DF8551A2A21A92AF2B
:013CAB00FF19
:013CAC0022F5
:103E0500A2AF921AC2AF8C838D82EF12206C43A2AF
:0C3E15002012206E53A2DFA21A92AFFF11
:013E2100227E
:023D59008F4B8E
:103D5B00A2AF921AC2AFE4F5838D82740612206C67
:103D6B00E54B43A22012206E53A2DFA21A92AF7F23
:013D7B000146
:013D7C002224
:023D7D008F4B6A
:103D7F00A2AF921AC2AFE4F5838D82740A12206C3F
:103D8F00E54B43A22012206E53A2DFA21A92AF7FFF
:013D9F000122
:013DA0002200
:101E9500A907E7FFA805EF93C3966008403B74FCCC
:101EA5002FFF80F00F08EF93C3966008402B74FB5B
:101EB5002FFF80E00F08EF93C3966008401B74FA6C
:101EC5002FFF80D00F08EF93D3966008400B74F96D
:101ED5002FFF80C01F1F1F1F1FEF54FEF80303F7BE
:101EE500E893FC08E893FD08E893FE08E893FF22D1
:101EF50009E993C39D6008402974FB29F980F1091C
:101F0500E993C39E6008401A74FA29F980E209E949
:101F150093D39F6008400B74F929F980D3191919D7
:101F25001919E9C313C313FF22740093F8ECC3987E
:101F35004024701F740193F8EDC398401970147410
:0E1F45000293F8EEC398400E7009740393F8EF
:101F5300EFC39840037F00227F0122EDF8E6F008EB
:101F6300A3DFFA22EDF8E0F608A3DFFA22E0A36389
:101F7300A201F0A363A201DFF475A2002263A20110
:101F8300F0A363A20122E0A363A201F0A363A20171
:101F9300E0A363A201F0A363A201E463A201F0A39F
:101FA30063A201DFE175A20022E0A363A2016DFE3B
:101FB300936CFDEE058393FC158363A201DFEA7541
:101FC300A200227F00E493A363A201F00F600CA39D
:101FD300E583C2E3F58363A20180EA75A20022E0F0
:101FE300A363A201F0A3E583C2E3F58363A201DF48
:101FF300EE75A20022E0A363A201F0A3E583C2E48D
:10200300D2E3F58363A201DFEC75A20022E0A363B0
:10201300A201F0A3E58344F8C2E5F58363A201DFDF
:10202300EC75A20022E583C2E3F583E0A363A2017A
:10203300F0A363A201DFEE75A20022E583C2E4D21E
:0A204300E3F583E0A363A201F0A31C
:10204D0063A201DFEC75A20022E58344F8F583E07D
:10205D00A363A201F0A363A201DFEE75A20022F932
:10206D0022C002C004C00612FFF0D006D004D00278
:01207D002240
:103A84002043616E457247495400200A0045727212
:103A94004C656E43616E21000A002043616E4572DD
:103AA40072434821000A205265714572722100C296
:103AB40000C201C202C203C204C205C206C2070098
:103AC40000000000000000000000000000000000F2
:103AD40000000000000000000000000000000000E2
:013AE40000E1
:10269900E59B541F6020200B1A7E3A7F84122D1D62
:1026A900E59B541FFF7E007D03122EEB7E3A7F8E41
:1026B900122D1DE4F59BE5BA30E010E4F5B375B1D0
:1026C90080F5B2D216F53A9067DAF0E5CFF47003E7
:1026D9000227E3754D01E4F54CE5CFF4554D700340
:1026E9000227D1E54CC454F0F5B1E5B2547F64201A
:1026F90060030227A2E5B3540FF52C85BC28E5BD7C
:10270900541FFF131313541FFFE5BD54E044184F22
:10271900F529E5BDC43354E0FFE5BE131313541F77
:102729004FF52AE5BEC43354E0FFE5BF1313135434
:102739001F4FF52B85A32D85A32E85A32F85A330A8
:1027490085A33185A33285A33385A334E4F5B2206B
:10275900110FE528547EB5280843BDF875B350809C
:102769000375B3D0301108E52830E7037F0022E56F
:102779002CD39408401D200B177E3A7F91122D1DF2
:10278900AF2C7E007D03122EEB7E3A7F9C122D1D0D
:102799007F0022E52C2405FF22E5B2549F60232007
:1027A9000B207E3A7F9E122D1DAFB27E007D031253
:1027B9002EEBAFB37E007D03122EEB7E3A7F9C1287
:1027C9002D1DE4F5B275B3D0E54D25E0F54D054C69
:0C27D900E54CC3940850030226E27F0088
:0127E50022D1
:103A22009066A4E0C39464505675B180E4F5B3F592
:103A3200B28528BCE52AC4135407FFE52954E04F98
:103A4200F5BDE52A33333354F8FFE52BC41354078D
:103A52004FF5BEE52B33333354F8F5BF852DA385DF
:103A62002EA3852FA38530A38531A38532A3853369
:103A7200A38534A3E52C540F2450F5B3753A0AC23A
:023A820016220A
:1030A70075B190E5B220E613200B107E3A7FA91286
:1030B7002D1DAFB27E007D03122EEBE4F5B3F5B202
:1030C700E50F30E615E4F50F906A00E02402F0E022
:1030D700903AB3937004906A00F07427250FF58235
:1030E700E43467F583E0702D906A00E0FFC3132492
:1030F700E7F582E43469F583E07005430F808015B6
:10310700E4F50F906A00E02402F0E0903AB3937080
:1031170004906A00F0E50F30E721906A00E0FF9025
:103127003AB393F5BCE4F5BDEFA393FF33333354C0
:10313700F8F5BE75BF78430F4080367427250FF525
:1031470082E43467F583E0F5BC75BD807428250FEC
:10315700F582E43467F583E0FF33333354F8F5BE83
:1031670075BF78050F050FE50FC394324003E4F5EB
:053177000F75B35022AA
:09002600EF6003C29622D296227B
:1037660043AB01C2E8C2EAE4FFEFC454F0F5B1C3CB
:10377600EF64809488500575B3D08003E4F5B3E414
:10378600F5B2F5BCF5BDF5BEF5BFF5C4F5C5F5C694
:10379600F5C7F5A3F5A3F5A3F5A3F5A3F5A3F5A33F
:1037A600F5A30FBF0EC39066A4E0FE25E0F5B47541
:1037B600B50C75B66C75A11275AB0275C13E75C3B5
:1037C600FF75C203E4906A00F0750F80FF7F1990C1
:1037D60069E7E4F0A3DFFCE4FF7F32906727E4F0BB
:0337E600A3DFFC62
:0137E90022BD
:101C96003E2A2C312CCFE0F0E0ECE5F2F0FB20E41C
:101CA600E8F1EFE5F2F7E5F0F1EAE8E3EE20F9E82E
:101CB600F2E00A003E4C2C4930312C256C752CD1B3
:101CC600EAEEF0EEF1F2FC20EEE1ECE5EDE020EDDF
:101CD600E020F8E8EDE52052533438352C31323027
:101CE600302C323430302C343830302C39363030D9
:101CF6002C31393230302C33383430302C353736BD
:101D060030302C3131353230300A003E4C2C4930DF
:101D1600352C25732CD2E8EF20F9E8F2E02C3020A0
:101D26002D2053323030302C31202D20D2CA313183
:101D3600330A0030202D2053323030300031202D30
:101D460020D2CA313133003E4C2C4930322C257317
:101D56002C43EAEEF0EEF1F2FC20EDE020F8E8ED9F
:101D6600E52043414E2C30202D20353030EAE12845
:101D76003530EC292C31202D203530EAE12835305C
:101D860030EC292C32202D20D8E8EDE020EEF2EBC5
:101D9600FEF7E5EDE00A0030202D20353030EAE18F
:101DA600283530EC290031202D203530EAE1283560
:101DB6003030EC290032202D20D8E8EDE020EEF27C
:101DC600EBFEF7E5EDE0003E532C4930332C25625F
:101DD600752CCFE5F0E8EEE420E8EDE4E8EAE0F67D
:101DE600E8E820282A3130ECF129283C3235302920
:101DF6000A003E532C4930342C2562752CCFE5F071
:101E0600E8EEE420ECEEF0E3E0EDE8FF20282A31EE
:101E160030ECF129283C323530290A003C21003CBF
:101E26004930313D003C4930323D003C4930333D7C
:101E3600003C4930343D003C4930353D000A417391
:101E46004F55543A000A4970496E3A000A546F4396
:101E5600414E3A00205265496E69742043414E0A4C
:101E6600002043414E283029203E20544F210A00AD
:101E7600D1F2E0F0F220F1EAE0EDE8F0EEE2E0ED9A
:0F1E8600E8FF0A000A4173796E634B65793A00F1
:103DC500E4F5D975DE31F5E9F5F9F5ECF5FCF5EE37
:103DD500F5FEF545F5479067D9F075D84075B740BC
:033DE500D2AE2239
:030033000223A9FC
:0F23A900C0E0C083C082C0D075D000C006C0079E
:1023B80030DC1D85FE6985EE6A74A1256AF56A74AC
:1023C800133569F569856AEC8569FCC2DC75DC49F9
:1023D80020DA0302251DA297929385FC6985EC6A91
:1023E8007442256AF56A74273569F569856AEC854A
:1023F80069FCE54514603414603E24FE7003022530
:10240800162404600302251B3097089067D9E0045E
:10241800F080059067D9E4F09067D9E0D3940A502A
:102428000302251BE4F0054502251B30970302250E
:102438001BD295054502251BE526C313F5263097C3
:10244800042480F5260547E5475407600302251B49
:10245800E547131313541FFF24DAF582E43468F5B3
:1024680083E526F0BF030675450002251BEF6406C9
:1024780070469068DEE0FF9068DBE0B5071D906865
:10248800DFE0FE9068DCE0B506119068E0E0FE90C1
:1024980068DDE0B5060575450080787545009068EB
:1024A800DBEFF09068DFE09068DCF09068E0E090A7
:1024B80068DDF0754718805BE547131313541F64F4
:1024C8000970469068E1E0FF9068DBE0B5071D9071
:1024D80068E2E0FE9068DCE0B506119068E3E0FE93
:1024E8009068DDE0B50605754503802775450090C1
:1024F80068DBEFF09068E2E09068DCF09068E3E079
:102508009068DDF0754718800A75450480057545A3
:0525180001C295C2DACA
:0D251D00D007D006D0D0D082D083D0E032DD
:10317C007BFF7A1C799612146E9069E5E0FEA3E051
:10318C00FFC3E49FFFE49EFEAB07FA3395E0F9F82A
:10319C007F007E8C7D0A7C00121A618F568E558DB5
:1031AC00548C537BFF7A1C79BA12146EE53F701461
:1031BC007553FF75541D7555397BFF7A1D791112A6
:1031CC00146E80127553FF75541D7555437BFF7A31
:1031DC001D791112146E9066A4E070127553FF7570
:1031EC00541D75559D7BFF7A1D794D12146E90669A
:1031FC00A4E0B40A127553FF75541D7555AC7BFFD2
:10320C007A1D794D12146E9066A4E0B46412755355
:10321C00FF75541D7555BB7BFF7A1D794D12146ECD
:10322C007BFF7A1D79CD853B5312146E7BFF7A1D83
:09323C0079F885385312146E2252
:103245007E1E7F221235D8EF4E70037F01227E1E2F
:103255007F251235D8EF4E6023123AE5A804A9055B
:10326500AA06AB077F007E8C7D0A7C00121A6112CC
:103275001AF39069E5EEF0A3EFF0800A9069E57422
:10328500FFF0A374B8F0E49066A4F07E1E7F2B12C5
:1032950035D8EF4E601B123E228F4BE54BB43106FD
:1032A5009066A4740AF0E54BB432069066A4746483
:1032B500F07E1E7F311235D8EF4E6007123AE58F4A
:1032C5003B8003753B647E1E7F371235D8EF4E6019
:1032D50007123AE58F38800375385AE4F53F7E1EAC
:1032E5007F3D1235D8EF4E600D123E228F4BE54BD8
:0832F500B43103753F017F00B5
:0132FD0022AE
:03002300022B2885
:0D2B2800C0E0C0F0C083C082C0D075D018DE
:102B3500309841C298AF9920120BEF64027035D2DC
:102B450012D291802F301707C217531F0F8016BF5F
:102B55000904D217801EBF030C853E43753E00C293
:102B650012C291800F74DB253EF582E43467F5834C
:102B7500EFF0053E209903022C20201303022C1EA2
:102B8500E53F706FE540B4FF0D7599020540754648
:102B950000D290022C1EE540B53D0BC212C29175C4
:102BA500990305408073E540D3953D400DC213D28E
:102BB50019E4FF120026C290805FE5466009F59989
:102BC5000540754600805274E52540F582E4346879
:102BD500F583E0F5466402600BE54664036005E5B0
:102BE50046B40905759909803085469905407546AD
:102BF500008026E540C3953D400DC213D219E4FF80
:102C0500120026C2908012D29074E52540F582E428
:0B2C15003468F583E0F5990540C29992
:0B2C2000D0D0D082D083D0F0D0E032C2
:1039BA00E4FF120026C213C219C212C217E4F5406C
:1039CA00F53DF53E9069E574FFF0A374F4F0E490D8
:1039DA0066A6F0F50F9066A4F0753B6475385A1226
:1039EA003245C2ADE4F5C9D2CDD2CCC2C9C2CAF5FC
:1039FA00CDF5CC9069E5E0F5CBA3E0F5CA85CBCD52
:103A0A0085CACCD29ED29CD2CAC2ACC298C299757F
:083A1A00B81075B710D2AC2200
:0100210022BC
:022C2B008F4CCC
:102C2D00E53F7003022CB890637CE0FF64086003FD
:102C3D00022D1C90637AE09067DBF090637BE0FEE1
:102C4D009067DCF0A3EFF09068E57472F0EEC45479
:102C5D00F0FFA3F090637DE09068E7F090637EE075
:102C6D009068E8F090637FE09068E9F0906380E011
:102C7D009068EAF0906381E09068EBF0906382E0F9
:102C8D009068ECF0906383E09068EDF0906384E0E1
:102C9D009068EEF0A37474F0A3EFF07F011200269C
:102CAD00753D0CE4F540750B018050E4FFFEEEC35D
:102CBD00954C5028747A2EF582E43463F583E0FD4B
:102CCD0074E52EF582E43468F583EDF074E52EF5A8
:102CDD0082E43468F583E02FFF0E80D2EFF4FF74A9
:102CED00E5254CF582E43468F583EFF07F011200A1
:102CFD0026E54C04F53D7540FFD299D213200B0DFE
:0F2D0D007E1E7F437C687DE5AB3D12291DC219F8
:012D1C002294
:103CE000300008C2009066A5E004F030130F906623
:103CF000A5E0D39414400BC213D2198005E490665A
:0F3D0000A5F0E50BD394034005D299E4F50B220F
:03001E00E4FF22DA
:103D0F00C28DC2AF438901C28C9066A4E0FF7007D9
:103D1F00F58A758CEE800AEFB40A06E4F58A758C85
:063D2F0070D28CD2AF221D
:103CAD00C28DC2AF438901C28C9066A4E0FF70142F
:103CBD00301809F58A758CDCC2188012758A667504
:103CCD008CFC800AEFB40A06E4F58A758CDCD28C84
:033CDD00D2AF2241
:103DA1009066A4E0C394645006123766123D0F1268
:103DB1000021D216E4F53A9067DAF0F525F549C20B
:043DC10018F542228D
:0227E600AB073F
:1027E800EB24FCF54B200B0B7E1E7F4B7C637D7628
:1027F80012291D906379E0641F6003022903906326
:1028080076E0B40117E544C39403400AE544D39441
:10281800FA500302291CAF4B122C2B2290637CE048
:10282800640870459067597442F0A37418F0906377
:102838007AE0FFC4540F90675BF0EFC454F0FF9048
:10284800637BE0FEC4540F2F90675CF0A37408F01C
:1028580090637D63A20190675E63A201FF121F70FF
:1028680075250DE4F537C2142290637CE0FFB40AA5
:102878001D9067597401F0A37418F0A37480F0A335
:10288800740AF0E4A3F0752505F537C21422EFB4F5
:102898000B1D9067597401F0A37418F0A37480F0AD
:1028A800A37409F0E4A3F0752505F537C21422EFE7
:1028B800B40D1D9067597401F0A37418F0A37480C7
:1028C800F0A3740BF0E4A3F0752505F537C21422C4
:1028D800EF6407703F90675904F0A37418F0A3746D
:1028E80080F0A3740CF0A37401F090637DE090670E
:1028F8005EF0752506E4F537C2142290637A63A268
:102908000190675963A201AF4B121F70854B25E4F4
:04291800F537C214B9
:01291C002298
:03002F008F4B22D2
:10176800208D030217F0C28D2016030218A9E52563
:10177800604C90675DE02405F54BE4F525E54BD317
:10178800940D4008D214123D0F0218A9906759E52C
:101798004B540FFF7D28121F67E52830E702D21847
:1017A800200B107E1E7F527C677D59E54B540FFB42
:1017B80012291D123D0F123A22D2140218A9E53C33
:1017C8006017906690540FFF7D28121F67123D0F17
:1017D800123A22E4F53C0218A99066A4E0C3946486
:1017E80050031230A7123D0F1226998F4BEF70034A
:1017F8000218A9123CADE4F542E548C3946E4003D3
:101808000218A92003030218A9E5286442706FE5AD
:101818002C7032E52AC454F0FFE52BC4540F2FF581
:1018280028E52BC454F0F529752A0874A72548F52E
:1018380082E43466F58374032548F5487D287F03E0
:10184800121F5E805C74A72548F582E43466F58330
:10185800E54B2548F5487D28AF4B121F5E300D41FA
:10186800C3E548954BFFE49400FE74A72FF58274F6
:10187800663EAF82FEE4FBAD4B122FCC8023E528F9
:10188800B44206E52B6402601874A72548F582E483
:101898003466F583E54B2548F5487D28AF4B121F84
:1018A8005E300E1030000B9066A4E0C394645002C2
:1018B8000542C20E200203021A21E53A6031D39490
:1018C800014004153A80289067DAE004F0E0D394E8
:1018D80003400D200B077E1E7F5A122D1D123DA1BD
:1018E800200B077E1E7F67122D1DE4F53AD216E500
:1018F80044C394FD5002054420AE5520B33DE54451
:10190800D394FA4009E54494FE5003E4F544E544D1
:10191800640F60030219DD200B077E1E7F76122DEF
:101928001D90637A74FFF0A3F0A37409F07F03128B
:101938002C2B123DC5E4F5440219DDE544C3940A95
:101948004008E544F460030219DD7544FD0219DD21
:10195800E54564037064200B0D7E1E7F8A7C687DDC
:10196800DB7B0912291D300D159068DB7443F0E408
:10197800A3F0A3F07E687FDBFB7D06122FCC20B39B
:10198800239068DEE090637AF09068DFE090637BF4
:10199800F0A37418F09068E0E090637DF07F041283
:1019A8002C2B801190637A74FFF0A3F0A3740DF0D0
:1019B8007F03122C2BC2AE7544FFE544B4FA16908F
:1019C800637A74FFF0A3F0A3740DF07F03122C2B3D
:1019D800C2AE7544FFE53C703E0539E539B53818A7
:1019E8009066907401F0A37408F0A37480F0A37457
:1019F80008F0E4A3F0753C05E539B53B1AE4F53980
:101A080090669004F0A37408F0A37480F0A37407A0
:0C1A1800F0E4A3F0753C05C202123CE0B3
:011A2400229F
:10395000E5436033E4F54390647604F0A37403F028
:1039600090667BE0906478F0A3741FF09067DBE0D2
:1039700090647AF09067DCE090647BF09067DDE023
:1039800090647CF07F0122E548602CE4906476F03E
:10399000A3E548F090667BE0906478F0A3741FF094
:1039A0009066A763A20190647A63A201AF48121FD8
:0A39B00070E4F5487F01227F002239
:103E3C00301405C2147F022230190CC219E53F6000
:0A3E4C00037543037F03227F002269
:0100220022BB
:063E6D00E4F548F52522F2
:0100320022AB
:10344A000208EFE493A3F8E493A34003F68001F2A1
:10345A0008DFF48029E493A3F85407240CC8C33383
:10346A00C4540F4420C8834004F456800146F6DF52
:10347A00E4800B0102040810204080903E66E47E3E
:10348A00019360BCA3FF543F30E509541FFEE49347
:10349A00A360010ECF54C025E060A840B8E493A30E
:1034AA00FAE493A3F8E493A3C8C582C8CAC583CA39
:1034BA00F0A3C8C582C8CAC583CADFE9DEE780BEF1
:013E6C000055
:101A250075F008758200EF2FFFEE33FECD33CDCC78
:101A350033CCC58233C5829BED9AEC99E5829840FB
:101A45000CF582EE9BFEED9AFDEC99FC0FD5F0D6D8
:101A5500E4CEFBE4CDFAE4CCF9A88222B800C1B902
:101A65000059BA002DEC8BF084CFCECDFCE5F0CB40
:101A7500F97818EF2FFFEE33FEED33FDEC33FCEB79
:101A850033FB10D703994004EB99FB0FD8E5E4F934
:101A9500FA227818EF2FFFEE33FEED33FDEC33FC21
:101AA500C933C910D7059BE99A4007EC9BFCE99A15
:101AB500F90FD8E0E4C9FAE4CCFB2275F010EF2F5A
:101AC500FFEE33FEED33FDCC33CCC833C810D7075A
:101AD5009BEC9AE899400AED9BFDEC9AFCE899F895
:0E1AE5000FD5F0DAE4CDFBE4CCFAE4C8F92228
:0E1AF300C3E49FFFE49EFEE49DFDE49CFC2204
:101B0100EB9FF5F0EA9E42F0E99D42F0E89C45F03A
:011B110022B1
:0C1B1200ECF0A3EDF0A3EEF0A3EFF02246
:101B1E00A8828583F0D083D082121B35121B35121A
:101B2E001B35121B35E473E493A3C583C5F0C5833F
:101B3E00C8C582C8F0A3C583C5F0C583C8C582C811
:011B4E002274
:10140C00E55F2453F8E6055F2278503021027853CB
:10141C00E475F001121BF6021B4F201AEB7F2ED243
:10142C001A8018EF540F2490D43440D4FF301E0B84
:10143C00EF24BFB41A0050032461FFE5606002156D
:10144C00600563E5637002056230210D7850E47528
:10145C00F001121BF6EF021B95023BF87403D2212C
:10146C008003E4C221F55F8B508A518952E4F56008
:10147C00F562F563E56060077F2012144780F5750F
:10148C0061FFC21BC21AC21CC21DC21FC220C222D3
:10149C00121415FF700D3021057F00121458AF6324
:1014AC00AE6222B4255FC2D5C21E121415FF24D021
:1014BC00B40A00501A75F00A786030D50508B6FFEA
:1014CC000106C6A426F620D5047002D21D80D924AC
:1014DC00CFB41A00EF5004C2E5D21E021658D21B2C
:1014EC0080C6D21A80C0D21C80BCD2D580BAD21F82
:1014FC0080B47F20121447201C077401B560004093
:10150C00F112140CFF121447021480D222D2208044
:10151C009512140CFB12140CFA12140CF94A4B70A1
:10152C000679297A177BFF201C2EE560602A7E0045
:10153C008E82758300121B6860060EEE656170F07A
:10154C00C2D5EBC0E0EAC0E0E9C0E0EE12169FD0D5
:10155C00E0F9D0E0FAD0E0FB121B4FFF60AAEBC021
:10156C00E0EAC0E0E9C0E0121447D0E02401F9D071
:10157C00E03400FAD0E0FBE5610460DCD561D98091
:10158C00877BFF7A16799BD21C809C79108002791C
:10159C0008C220C2228008D2D5790A8004790AC2F6
:1015AC00D5E561047002F561E4FAFDFEFF12140C3E
:1015BC00FC7B08201B1312140CFD7B10301A0A1232
:1015CC00140CFE12140CFF7B20EC3382D592D550F8
:1015DC0013C3E4301A069FFFE49EFEE4201B039D18
:1015EC00FDE49CFCE4CBF8C21BEC700CCFCECDCC54
:1015FC00E824F8F870F38017C3EF33FFEE33FEEDF9
:10160C0033FDEC33FCEB33FB994002FB0FD8E9EBD9
:10161C00301B05F8D0E0C448B21BC0E00AEC4D4EBC
:10162C004F78207B0070C2EAB5610040BCC0E0126C
:10163C0016A1D0F0D0E0201B04C4C0E0C4B21BC083
:10164C00F0121430D0F0D5F0EB021480121C5515AA
:10165C001D5315975814EE4C14EA42159B4F15A3C5
:0F166C004415A34915034315A955158D46158D32
:10167B0045158D4717495014F22D14F62E15192BBD
:10168B0014FA2315172017322A14B248000015112B
:10169B003F3F3F00790AA2D5201D14301F09B91016
:1016AB00020404B9080104A2D52020025001042031
:1016BB001C68921CB560005034C0E07F20301D19AF
:1016CB007F30A21C7220721F500F1216F8C21CC260
:1016DB0020C21FC2227F30800F301F03E9C0E012EF
:1016EB001447301F03D0E0F9D0E0B560CC301F17A2
:1016FB007F30B9100C1214477F58301E077F78804B
:10170B0003B90803121447301C057F2D0214477FC1
:10171B00202022F87F2B2020F322921C80CF286ED2
:10172B00756C6C2900D21B12140C301BF8C21B7881
:10173B006030D50108F60214B22D504349581214EB
:10174B000C2403B405004001E490174493121438A1
:0D175B00743A121438D21D756004021597FF
:10207E008B4C8A4D894EE4F558F557F556F555F5C6
:10208E0053F554E5504551454F6012EBC0E0EAC0A0
:10209E00E0E9C0E0AB4FAA50A951121C06AB4C05AB
:1020AE004EE54EAA4D7002054D14F9121B4FF5590F
:1020BE00C394094007E559D3940D40E1E5596420D6
:1020CE0060DBE559B42D054354038016E559B42B56
:1020DE0005435401800C74FF254EF54E74FF354DAB
:1020EE00F54DE55260046410703FAB4CAA4DA94EFD
:1020FE00121B4F64306009E552702E75520A80290A
:10210E00900001121B68FF64786004EFB45813430B
:10211E0054017552107402254EF54EE4354DF54DB1
:10212E008007E5527003755208AB4C054EE54EAA7A
:10213E004D7002054D14F9121B4FF559C3946140B1
:10214E000AE559D3947A50035359DF74D02559F5C3
:10215E0059C3940A400CE5599411406D74F92559F0
:10216E00F559E559D39552506043540185585D8514
:10217E00575C85565B85555AAF527E00E4FCFDAB2D
:10218E0058AA57A956A855121BA7C8ECC8C9EDC91D
:10219E00CAEECACBEFCBE4FCFDFEEB2559F558EEAB
:1021AE003AF557ED39F556EC38F555AF58AE57AD03
:1021BE0056FCAB5DAA5CA95BA85AD3121B01500357
:1021CE00022137435404022137E55420E003E48012
:1021DE002DE5504551454F601EAB4CE54E24FFF9A1
:1021EE00E54D34FFFAEBC0E0EAC0E0E9C0E0AB4FEA
:1021FE00AA50A951121C06E55430E20774FFFFFEE7
:10220E00FDFC22E554AF58AE57AD56AC5530E10348
:04221E00021AF3228B
:101B4F00BB010689828A83E0225002E722BBFE0294
:091B5F00E32289828A83E49322C7
:101B6800BB010CE58229F582E5833AF583E0225032
:101B780006E92582F8E622BBFE06E92582F8E2227C
:0D1B8800E58229F582E5833AF583E4932296
:101B9500BB010689828A83F0225002F722BBFE012F
:021BA500F32229
:101BA700E88FF0A4CC8BF0A42CFCE98EF0A42CFCDD
:101BB7008AF0EDA42CFCEA8EF0A4CDA8F08BF0A45B
:101BC7002DCC3825F0FDE98FF0A42CCD35F0FCEBBA
:101BD7008EF0A4FEA9F0EB8FF0A4CFC5F02ECD397F
:0F1BE700FEE43CFCEAA42DCE35F0FDE43CFC22EC
:101BF600FAE6FB0808E6F925F0F618E6CA3AF622F0
:101C0600BB011A89828A83D0F0D0E0F8D0E0F9D0FF
:101C1600E0FAD0E0FBE8C0E0C0F0021C845016E910
:101C2600F8D083D082D0E0F9D0E0FAD0E0FBC082D1
:101C3600C083021C7BBBFE16E9F8D083D082D0E0BD
:0F1C4600F9D0E0FAD0E0FBC082C083021C8D22EF
:101C5500D083D082F8E4937012740193700DA3A31E
:101C650093F8740193F5828883E473740293686032
:061C7500EFA3A3A380DF32
:091C7B00EBF608EAF608E9F6228E
:091C8400EBF0A3EAF0A3E9F02261
:091C8D00EBF208EAF208E9F22288
:00000001FF
